:100000000C9434000C9451000C9451000C94510049
:100010000C9451000C9451000C9451000C9451001C
:100020000C9451000C9451000C9451000C948D01CF
:100030000C9451000C9451000C9451000C945100FC
:100040000C9451000C9451000C9451000C945100EC
:100050000C9451000C9451000C9451000C945100DC
:100060000C9451000C94510011241FBECFEFD4E02A
:10007000DEBFCDBF11E0A0E0B1E0ECE5F4E002C0EE
:1000800005900D92A430B107D9F711E0A4E0B1E0DA
:1000900001C01D92AE30B107E1F70E94B7010C9488
:1000A0002C020C9400002CEB37E004C0F9013197CE
:1000B000F1F701970097D1F70895E09106018823A1
:1000C00071F4E60FE370E093060190910701F0E010
:1000D000E050FF4F80818295807F9F700DC080919E
:1000E0000501680F63706093050180910701F0E0DE
:1000F000E050FF4F807F9081892B80930701809192
:1001000007018BB90895DF92EF92FF920F931F932F
:1003F0003197F1F70197D9F72196CA30D10541F726
:10040000509A519A529A539A549A559A569A579A80
:1004100080E061E00E945D0081E061E00E945D009B
:1004200081E06CE341E00E94830084E064E04CEBF7
:1004300052E024E630E00E941701CCEBD7E082E3E3
:1004400090E064E00E94D60084E893E0FE013197DA
:0C045000F1F70197D9F7F3CFF894FFCF34
:04045C0005060A097E
:00000001FF
